:0400000080316028C3
:100008007E14803120001508F000F1017008F2001C
:100018007108F3000B1C1128122857280B10270011
:10002800161F172818282A2820000D1B1C281D28F1
:100038002A2827001613200095012708031D2528C4
:10004800262857288C31E624803157282700161F88
:100058002E282F28572820000D1F332834285728EA
:100068002700161306302000270203183C283D28D5
:1000780057287208F0002708CA3E860087017008D2
:1000880081000130F0007008A70706302706031D1D
:100098004E284F2857288C31E02480310130F00059
:1000A80070082000A6000B1D5A285B285E280B113B
:1000B8002000A7017E100900803162288731FE27C1
:1000C8008031C6008731FF278031C700F601F7016C
:1000D800F801F901203084000030850016308C3199
:1000E800EB248031CA308400003085001B308C310D
:1000F800EB2480317E1020008031822885317525DF
:10010800803131308D31ED2580312C308D31ED2528
:100118008031D2308E3147268031A2308731142782
:100128008031AC30873114278031B6308731402791
:100138008031C0308731402780318D318A25803128
:100148008D31552580318D319825803187316C2747
:10015800803175082000A1007408A0007A302102BF
:10016800123003192002031CBA28BB28C5288D3178
:100178008A2580312000A001A1010130C60000308D
:10018800C7004708B7004608B6007D30B800003001
:10019800B9008E31B9268031200037082100A1002E
:1001A800200036082100A00084319A248031C03014
:1001B8002000C5004508BC00B6308E31FA268031D3
:1001C800AC302000C5004508BC00A2308F31422762
:1001D800803185312F2580318F31662780318D31EF
:1001E8003D2580310130F6000030F700B6302000A0
:1001F800C5004508C300A230813185218031023015
:10020800F6000030F700C0302000C5004508C300E4
:10021800AC308131852180318E310026803120003B
:100228003908C500C50DC50D22000C08200045067B
:10023800FB39450622008C00F81D23292429402972
:1002480005302000B6000030B7004708B90046085E
:10025800B8008631AE268031200036083704031DE9
:100268003629372940298D317C258031843137243E
:1002780080318D3155258031200026080319452904
:1002880046296229A601A201A301F8194C294D2982
:100298005E298431E72480318D317C258031A0307E
:1002A8000032890B54298431372480318D3155250A
:1002B80080316F298431E72480316F29013023028E
:1002C800F4300319220203186A296B296F290130B7
:1002D800A2070030A33D87316C2780312100210817
:1002E8007502031D792920087402031C7C297D29C5
:1002F8006F2901302000C6070030C73DA72880318C
:1003080060282000C40043088531B92581312000C8
:100318003E083F04031991299229392A8F311E2753
:1003280081317408750403199A299B29CD29200065
:1003380043088731BF278131740875040319A5293B
:10034800A629B9298E31152681318E312E26813183
:1003580000308F31D927813100308E319B26813191
:1003680001308E317D268131802A8E3115268131EA
:100378008E312E26813101308F31D92781310030DD
:100388008E319B268131210054088E317D268131A2
:10039800802A200043088731BF27813174087504FB
:1003A8000319D729D829EB298E31152681318E31A9
:1003B8002E26813100308F31D927813100308E319E
:1003C8009B26813101308E317D268131802A8F3103
:1003D8008B278131200039083A04031DF429F529B7
:1003E800082A8E31D92681318E312E26813100306E
:1003F8008F31D927813100308E319B2681310130F0
:100408008E317D268131802A8631792681318F315E
:100418008B278131200039083A040319142A152A38
:10042800252A8E312E26813100308F31D92781310E
:1004380000308E319B26813101308E317D2681310D
:10044800802A8E31152681318E312E268131013058
:100458008F31D927813100308E319B26813121009F
:1004680054088E317D268131802A440887319627A9
:100478008131740875040319422A432A462A8531B2
:10048800FD2581318F31B2278131200039083A04A6
:1004980003194F2A502A622A8E31152681310030DD
:1004A8008F31D9278131210052088E319B26813125
:1004B800210053088E317D268131802A8E31152600
:1004C80081318E312E26813100308F31D92781310B
:1004D80000308E319B268131200043088731BF27A9
:1004E800813174087504031D7A2A7C2A01307D2A1B
:1004F80000308E317D26813108002000BB00740851
:1005080075040319882A892ADA2A3B08023E8600DC
:100518008701403FB600413FB7003B08860087018E
:10052800403FB800413FB9003908803ABA0037085F
:10053800803A3A02031DA22A360838020318A52A6F
:10054800A62A232B20003B08860087010430810758
:1005580041310318810A3B0886008701403FB600F5
:10056800413FB7003B08043E86008701403FB80082
:10057800413FB9003908803ABA003708803A3A0250
:10058800031DC82A360838020318CB2ACC2A232B85
:1005980020003B08063E860087013B08083E840091
:1005A8008501403F803F413F813F232B3B08860028
:1005B8008701403FB600413FB7003708803AB8008E
:1005C80080303802031DEA2A01303602031CED2A66
:1005D800EE2A232B20003B0886008701FC30810788
:1005E8004131FF30813D7F313B08063E860087015F
:1005F800403FB600413FB7003B0886008701403FB7
:10060800B800413FB9003908803ABA003708803A43
:100618003A02031D112B360838020318142B152B28
:10062800232B20003B08043E860087013B08083E38
:1006380084008501403F803F413F813F232B0800D4
:100648002000C3004308043E8D31622583317408BD
:100658007504031D302B312B322BBF2B20003D0896
:10066800F5003C08F4004308043E86313B268331FC
:1006780075082000C0007408BF004308033E8600C8
:10068800870101080319492B4A2B692B3F084004AD
:1006980003194F2B502B692B4308043E8D316F25CE
:1006A800833120004308860087018101430A8600C0
:1006B800870181014308023E8600870181014308C2
:1006C800033E860087018101BF2B4308043E8D311C
:1006D8002725833120003708C2003608C1000330BF
:1006E8004202E83003194102031C7B2B7D2B0130A9
:1006F8007E2B0030BE004308860087013E0881003B
:10070800E830B6000330B7004208B9004108B80025
:100718008631AE268331013020003702F4300319C8
:100728003602031C982B9A2B01309B2B0030BE00FD
:10073800430A860087013E088100F430B600013084
:10074800B7004208B9004108B8008631AE268331A7
:10075800013020003702903003193602031CB52BF4
:10076800B72B0130B82B0030BE004308023E86008C
:1007780087013E08810008002000C00021004A08C7
:100788002000B600B7013708B90040083602B800A3
:10079800031CB903B91BD12BD22BDB2B400821003A
:1007A8004A022000BC00BD01031CBD03F02B210040
:1007B8004A082000B600B7013708B90040083602D9
:1007C800B800031CB903B809B909B80A0319B90A6A
:1007D8003808BC003908BD003C08B6003608BA0025
:1007E80021004B082000B600B7013708B9004008BF
:1007F8003602B800031CB903B91B032C042C152CB2
:1008080021004B082000B600B7013708B90040089E
:100818003602B800031CB9033808BE003908BF0007
:100828002A2C21004B082000B600B7013708B90070
:1008380040083602B800031CB903B809B909B80A58
:100848000319B90A3808BE003908BF003E08B600C7
:100858003608BB003B083A02031C332C352C013008
:10086800362C00300800F81D3A2C3B2C6C2C01303B
:100878008631E326843100308631E3268431210035
:100888005208031D482C4A2C01304B2C003086316D
:10089800E326843121005308031D532C552C0130C5
:1008A800562C00308631E326843121005408031D7C
:1008B8005E2C602C0130612C00308631E3268431B7
:1008C80022000E0D0E0D01398631E3268431992C54
:1008D80001308631E326843100308631E3268431C5
:1008E8008E3100268431200039083A04031D7D2CFE
:1008F8007F2C0130802C00308631E32684318D3105
:10090800C725843174087504031D8B2C8D2C013088
:100918008E2C00308631E326843100308631E32680
:10092800843100308631E3268431080012302000FB
:10093800B6007A30B7002108B9002008B80086311F
:10094800AE26843120003708BD003608BC00F81DEB
:10095800AE2CAF2CC12C3D08803ABA00BD303A020B
:10096800031DB82C0A303C02031CBB2CBE2C2200F1
:100978008E17C02C22008E13E62C01302302F4308F
:1009880003192202031CC92CCA2CE62CBB013D0802
:10099800803ABA00BD303A02031DD42C0A303C021A
:1009A8000318D72CD82CDF2C2000C61DDC2CDD2CFE
:1009B800DF2CBB01BB0A20003B0C2200031C8E135A
:1009C80003188E1708000630200027060319ED2C9F
:1009D800EE2CEF2C2E2DF819F22CF32C1A2D2100C9
:1009E8004C088331C0238431F40074082100D200FC
:1009F8004D088331C0238431F40074082100D300EA
:100A08004E088331C0238431F40074082100D400D7
:100A18004F088331C0238431F400F40CF40C220015
:100A28000E0874067F3974068E002C2D21004C08A0
:100A38008331C0238431F40074082000A50021000C
:100A48004D088331C0238431F40074082000A400C9
:100A58002000A7010800F81D322D332D702D8E318E
:100A680000268531200039083A04031D3C2D3D2D10
:100A7800582D8D310A25853174087504031D452DBF
:100A8800462D582D8D31C725853174087504031DF1
:100A98004E2D4F2D582D8D31012585317408750443
:100AA8000319572D582D622DA0302000B9000F30A2
:100AB800BA00D2308E3160268531662DD2308D3124
:100AC8001325853104302000BC000030BD00D23031
:100AD800833124238531742DD2308D31132585310E
:100AE8000800210019088739683899001908FC3965
:100AF800023899009913951338308C003830270044
:100B08008C00383024008C00C03021008D00F0307B
:100B180027008D00C03024008D00783021008E0021
:100B2800783027008E00783024008E0023008C0156
:100B38008D018E0121009D0126008C018D018E0101
:100B48008D31492585318D311D2585318C31F12433
:100B580085318D313225853100308D31B52585318E
:100B68008B150B178B178B1708002000C2008F31CD
:100B7800B2278531200039083A040319C42DC52D40
:100B8800EF2D42088731BF27853174087504031D8E
:100B9800CE2DCF2DEF2D2000BE01BF01FC2D200052
:100BA800291ED72DD92D0130DA2D0030C000C10102
:100BB8004008BE004108BF00FC2D781FE42DE62D3B
:100BC8000130E72D00302000C000C1014008BE0000
:100BD8004108BF00FC2D7708003A0319F42DCF2DEA
:100BE8007608013A0319D32D033A0319E12DCF2DC5
:100BF800080031308D31DA25853174087504031900
:100C0800062E072E2D2E2C308D31DA2585317408CD
:100C180075040319102E112E2D2EA0302000B900B6
:100C28000F30BA00D2308E31602685312D2E7030CB
:100C3800F4001730F50031308731E82785313A2E36
:100C48007030F4001730F5002C308731E8278531F3
:100C58003A2E7708003A0319322E3A2E7608013ACE
:100C680003191B2E033A0319242E3A2E08002000DC
:100C7800BB003B08860087010108031D442E452E52
:100C8800482EF401F501782E3B0A86008701403F83
:100C9800B600413FB7003B08033E86008701740851
:100CA800810741317508813D7F31403FB800413FA0
:100CB800B9003908803ABA003708803A3A02031D69
:100CC800672E3608380203186A2E6B2E6C2E452EB6
:100CD80020003B08033E860087010030C03FC13F2B
:100CE8000130F4000030F5000800A02E0430F400B4
:100CF8000030F500E03086313B26863174087504F3
:100D08000319872E882EAD2EE0308D316F25863160
:100D1800AD2E0430F4000030F500DB3086313B2680
:100D280086317408750403199A2E9B2EAD2EDB307C
:100D38008D316F258631AD2E7708003A0319A52E1F
:100D4800AD2E7608013A03197A2E033A03198D2E2F
:100D5800AD2E08002000360837040319B42EB52E2E
:100D6800DE2EF501F50AC12E0130B635B70D890B17
:100D7800B92E0130F4007408F507B71FC42EC52E2C
:100D8800B82E37083902031DCB2E36083802031C4B
:100D9800CE2ECF2ED32E3608B8023708B93B0130F5
:100DA800B736B60C890BD42E0130F502031DDD2EA3
:100DB800DE2EC52E3908B7003808B6000800200016
:100DC800B6003608031DE92EEA2EEF2E0A30B700CA
:100DD8000030B800FB2E1430B7000030B800FB2EEE
:100DE80022000D13FF302000B707FF30B83D370849
:100DF8003804031D002F012FF42E1430B7000030E3
:100E0800B8000D2F22000D17FF302000B707FF3064
:100E1800B83D37083804031D122F132F062F08007A
:100E2800F4007408860087010030C03FC13F740891
:100E3800023E860087011E30C03F0030C13F740863
:100E4800043E860087011430C03F0030C13F74085B
:100E5800063E860087010A30C03F0030C13F740853
:100E6800043E860087017408083E84008501403FDF
:100E7800803F413F813F0800F400740886008701E5
:100E88000030C03FC13F7408023E860087010A3027
:100E9800C03F0030C13F7408043E86008701073018
:100EA800C03F0030C13F7408063E86008701043009
:100EB800C03F0030C13F7408043E860087017408B3
:100EC800083E84008501403F803F413F813F080044
:100ED80020001708B600B7013608BB003708BC0069
:100EE8001608B600B7013608B9003708BA0017085F
:100EF800B600B7013C083706031D842F3B083606A9
:100F0800031D872F882F6C2F3C08B7003B08B600BD
:100F18003608B700B60139083604F4003A08370431
:100F2800F50008002000BD003D0886008701403F0D
:100F3800B600413FB7003D08083E86008701403FA4
:100F4800B800413FB9003908803ABA003708803AFA
:100F58003A02031DB12F36083802031CB42FB62FEE
:100F68000130B72F00302000BB00BC013B08F40063
:100F78003C08F50008002000BD003D0886008701F8
:100F8800403FB600413FB7003D08083E8600870154
:100F9800403FB800413FB9003908803ABA003708E5
:100FA800803A3A02031DDA2F36083802031CDD2F77
:100FB800DF2F0130E02F00302000BB00BC013B08D0
:100FC800F4003C08F50008002000B600360A860048
:100FD80087017408C03F7508C13F3608033E860084
:100FE80087010030C03FC13F360886008701810174
:080FF800810A080001340034F5
:1019C0008B120B1108008B120B11080020009501DF
:1019D0000B118B160800640080010131890BEC2C7F
:1019E0000034813020009B009A0191107F309C00D0
:1019F0000800200018107508970074089600181445
:101A0000080020002408B600B7013608F4003708A3
:101A1000F500080020002508B600B7013608F400DC
:101A20003708F5000800F5000130F4007508033EA2
:101A30008600870174088100080020009901F830B1
:101A40009700103096001110C13098000800F40083
:101A50007408033E86008701403F2000B600413FE6
:101A6000B70008000C303D00A1003C302500930079
:101A70004030910092019E01080021005208031D90
:101A8000422D442D0130452D00308D31A6258D315C
:101A9000080021009512151295111508F839033820
:101AA0009500200095010B1108002000A7012100DE
:101AB0000D1727000D1724000D170B102700141702
:101AC000151708002000B8003808860087010108B3
:101AD000B600B7013608F4003708F5000800F40036
:101AE00074088600870181017408033E860087011F
:101AF0000030C03FC13F08008C31E3248D31270006
:101B0000141315130B1022000D1721000D132200C2
:101B10000D1708000030F400F5008C31F9248D31E8
:101B20002000A001A1010130C6000030C70008005C
:101B300020000C08F4007408A9000D08F4007408D3
:101B4000A8000E08F4007408F8000800F4007403FC
:101B5000031DAB2DAC2DB02D0C303D00A100B42DDC
:101B60003D00A10122008E100800F4008B150B101F
:101B700074080319BC2DBD2DC22D2700141715178D
:101B80001613C62D27001413151316130800790811
:101B9000031DCB2DCC2DD22D20002B080319D12DC8
:101BA000D22DD72D0130F4000030F500D92DF401ED
:101BB000F50108002000B8003808860087010108F8
:101BC0000319E32DE52D0130E62D0030B600B701F5
:101BD0003608F4003708F5000800F400740A86009F
:101BE00087010030C03FC13F7408033E8600870173
:101BF0000030C03FC13F74088600870181010800A2
:101C000031308D3162258E3174082000BB0075089B
:101C1000BC002C308D3162258E31740820003B04CD
:101C2000B90075083C04BA000800202EE0308D3160
:101C30006F258E312D2EDB308D316F258E312D2E7F
:101C40007708003A0319252E2D2E7608013A03193C
:101C5000162E033A03191B2E2D2E0800392E313073
:101C60008D316F258E31462E2C308D316F258E3182
:101C7000462E7708003A03193E2E462E7608013A82
:101C800003192F2E033A0319342E462E0800F500AF
:101C90007508860087018101750A86008701810128
:101CA0007508023E8600870181017508033E8600A3
:101CB000870181017508043E8D31ED258E310800C4
:101CC0002000BB003B08033E8600870181013B08E2
:101CD000043E8D31DA258E31740875040319712E96
:101CE000722E7C2E20003A08F5003908F4003B08DB
:101CF000043E8731E8278E310800F4008D2E740CE5
:101D00002200031C0C1003180C149A2E740C2200D1
:101D1000031C8D1203188D169A2E7708003A0319AA
:101D2000922E9A2E7608013A03197F2E033A031950
:101D3000862E9A2E0800F400AB2E740C2200031C91
:101D40000E1103180E15B82E740C2200031C0D1270
:101D500003180D16B82E7708003A0319B02EB82EC6
:101D60007608013A03199D2E033A0319A42EB82EC2
:101D70000800F401F5012000361CBF2EC02EC42E31
:101D80003808F4073908F53D0130B835B90D890B2D
:101D9000C52E0130B736B60C890BCA2E360837046B
:101DA000031DD32ED42EBB2E7508B7007408B600C1
:101DB0000800EC2E3230F4000030F500E0308731BE
:101DC000E8278E31F92E3230F4000030F500DB3098
:101DD0008731E8278E31F92E7708003A0319F12E62
:101DE000F92E7608013A0319DA2E033A0319E32E85
:101DF000F92E08002000BF00F81EFF2E012F013031
:101E0000022F0030BD00BE013D08F4003E08F50081
:101E10003F08823181228E31781E0F2F112F013021
:101E2000122F00302000BD00BE013D08F4003E0826
:101E3000F5003C08823181228E310800342F790868
:101E40002000B600B7013608F4003708F500412F2E
:101E500020002B08B600B7013608F4003708F5005B
:101E6000412FF401F501412F7708003A0319392F6A
:101E7000312F7608013A03191F2F033A0319282F2F
:101E8000312F08002000BF00A91E472F492F013025
:101E90004A2F0030BD00BE013D08F4003E08F500A9
:101EA0003F08823181228F312000A81F582F5A2FDE
:101EB00001305B2F0030BD00BE013D08F4003E083C
:101EC000F5003C08823181228F3108000430F40093
:101ED0000030F500313086313B268F3174087504AF
:101EE0000319732F742F782F31308D316F258F3177
:101EF0000430F4000030F5002C3086313B268F3161
:101F0000740875040319852F862F8A2F2C308D3184
:101F10006F258F310800A42FE0308D3162258F317D
:101F200075082000BA007408B900B12FDB308D317C
:101F300062258F3175082000BA007408B900B12FEE
:101F40002000B901BA01B12F7708003A0319A92F6F
:101F5000A02F7608013A03198C2F033A0319962F04
:101F6000A02F0800CB2F31308D3162258F317508BD
:101F70002000BA007408B900D82F2C308D316225AA
:101F80008F3175082000BA007408B900D82F2000DE
:101F9000B901BA01D82F7708003A0319D02FC72FFB
:101FA0007608013A0319B32F033A0319BD2FC72F3F
:101FB0000800F500F22F750C2200031C8C1003188A
:101FC0008C147508F4007408F900FF2F750C2200BA
:101FD000031C0E1003180E147508F400740820007A
:101FE000AB00FF2F7708003A0319F72FFF2F760871
:101FF000013A0319DB2F033A0319E62FFF2F0800DC
:042000000434003470
:020000040001F9
:04000E00A4C9FBDEA8
:00000001FF
